:1000000015EF00F0EA6A060EE96EEF500DE0020E01
:10001000016E006A002EFED7012EFBD7970E006EF0
:10002000002EFED7EF2EF3D7000CF86AD09EEA6AB6
:10003000E96A700ED36ED350C150C00B0F09C16E68
:10004000070EB46EC150C00B0F09C16EC090C092B4
:10005000C094C09EC2809698C69A949E93809392B4
:10006000010EC66E000EC76ED190800ED56ECD6AA1
:10007000000ECA6E000ECB6E9484BD6AB76AB66A73
:10008000070EB46E9250926E060E006E002EFED7D2
:100090000000B450A19CB56A929A899A040E056E2C
:1000A000FA0E066EAFDF052EFBD7929A898A040EF0
:1000B000056EFA0E066EA6DF052EFBD7EDD7030000
:020000040030CA
:0E00000027C8390E0087A1000FC00FE00F4087
:00000001FF
